:0600000000008A01132834
:0800080009006D34613463341A
:10001000683469346E346534533474346134743400
:1000200065343D340034833083160313810083121A
:100030008B120B17313090006030F80077212028A8
:100040005320831203132B08F0002C08F1006430B6
:10005000F200F301812103193028F001F101332866
:100060000130F000F101F201F301812103193D2873
:10007000932083120313AB01AC012B08F0002C0872
:10008000F1000130F200F30188217008831203139C
:10009000AB007108AC002B211430F000F101962167
:1000A00021286300512883120313AB01AC01AD0179
:1000B000F001F1017008A000F001F1017008A40046
:1000C0000330F000F10170089F2171089F21831215
:1000D00003132008F000F1010130F200F301882140
:1000E000A821F300A821F200812103195A2803183E
:1000F0007E285A28700883120313A0000130F000F4
:10010000F1017008A7000230F000F1017008A800AA
:100110000830F000F1017008A9000930F000F10189
:100120007008AA0008000530F000F101BB2183121D
:1001300003132D08F000F10136220D30AF210A30F3
:10014000AF21831203132D08F000F1010030700677
:100150000319BB28013070060319D228023070063B
:100160000319E928033070060319FF2804307006CC
:100170000319162908000130F000F1017008A300EE
:100180000430F000F1017008A4000730F000F10124
:100190007008A5000530F000F1017008A6000130DC
:1001A000AD0008000230F000F1017008A300033038
:1001B000F000F1017008A4000830F000F1017008AF
:1001C000A5000130F000F1017008A6000230AD007A
:1001D0000800F001F1017008A3000530F000F10102
:1001E0007008A4000230F000F1017008A500093089
:1001F000F000F1017008A6000330AD0008000330E4
:10020000F000F1017008A3000830F000F10170085F
:10021000A4000130F000F1017008A5000430F000E6
:10022000F1017008A6000430AD0008000130F000B4
:10023000F1017008A3000430F000F1017008A4007F
:100240000330F000F1017008A5000230F000F10168
:100250007008A600AD01F001F1017008A000F000E7
:10026000F1017008233E84000008F000F1013230F3
:10027000F200F3016822F430F2000130F30088212B
:10028000700883120313A1007108A2002008F00077
:10029000F1017008273E84000008F000F1017008A9
:1002A000F4007108F5002108F0002208F100C322D3
:1002B0000330F000F10170089F2171089F21831223
:1002C00003132008F000F1010130F200F30188214E
:1002D000A821F300A821F200812103192D29031878
:1002E00076292D29700883120313A00008006730B7
:1002F0008316031399001815981683121816981769
:10030000080073087102031D0800720870020800DB
:100310007208F00773080318730AF1070800F00366
:10032000700FF10AF10370087104080083120313BF
:100330000B110B1D99298F21031D962908008B1382
:10034000F9007808840079088000F80A8B17080003
:100350008B13F8037808840000088B1708008312B9
:1003600003130C1EB12999000800700FF103F10A64
:10037000F00071040800C221003803190800AF2101
:10038000B521BB2971088A00700882000310F20DA4
:10039000F30DF40BC62908000310F30CF20CF40B58
:1003A000CC2908007208F0027308031C730AF102DA
:1003B0000800F601F701720873040319FF340130D5
:1003C000F40073080038031DF0297208013A031D78
:1003D000F0297008F6007108F700F001F10100340F
:1003E00070087104031DF5290034F31B002AF40A78
:1003F00074089F210130F400C621A821F400F529DA
:1004000072089F2173089F217608F2007708F30095
:1004100074089F210130F400C621A821F40072085D
:10042000F6007308F700A821F300A821F200D221FA
:1004300003181C2A88211D2A7614F403031900349A
:1004400074089F210130F400CC21A821F400002A77
:1004500000307104031D0800F0040800F009F109E0
:10046000B529F11F362A2D30AF212E22D001D1011E
:10047000D201D301D4010530F500F5030A30F200B2
:10048000F301D9215030750784007008303E800098
:100490007608F0007708F10028220319532A75081E
:1004A0000038031D3D2A0030F400503074078400EA
:1004B0000008031DAF21F40A7408053A031D552AEC
:1004C00008007008F60771080318710AF70708009A
:1004D000F601F701F401F50170087104031D712A9A
:1004E0000034720873040319832A721C7C2A612267
:1004F000031C7C2AF40DF50D0310F30CF20C031011
:10050000F00DF10D712A7608F0007708F100003443
:100510000310F20803190800F00DF10DF20B882A00
:1005200008007008F2007108F3000130F000F101DA
:10053000882208009122831603137008860471082C
:100540008704FF30F006F1067008831286057108F3
:1005500087057008831686057008870508009122B4
:10056000831203137008FA047108FB0470088604F0
:1005700071088704FF30F006F106700883168605BF
:100580007108870508007008F2007108F300FF3059
:10059000F000F100D2217008831203138E0071085D
:1005A0008F007408F000F101AF22831203130C10C6
:1005B0000C1CD82A0C107408F000F1019A220800D3
:00000001FF
